:10000000003065008D0108308E0020208F008F08A1
:100010000319192805148D0A1A208F0C03180510CE
:10002000031C05141A208E0B0D2805101A201A2007
:10003000032819280A308C0000008C0B1C2800347F
:100040000D088207483465346C346C346F342034C6
:1000500077346F3472346C3464340A340A340D34B7
:100060000034FF3FFF3FFF3FFF3FFF3FFF3FFF3FAA
:10400000FF3FFF3FFF3FFF3FFF3FFF3FFF3FFF3FC0
:00000001FF
